:020000040000FA
:10000000E228820700007E34093409340934FE34C2
:100010007F34493449344934B6343E344134413470
:100020004134A2347F344134413422349C347F340F
:1000300049344934C1347F340934093481343E347D
:10004000413449344934BA347F34083408340834EC
:10005000FF34FF34203440344034BF347F3408341C
:1000600014342234C1347F3440344034C0347F34BB
:1000700002340434083404340234FF347F3404344A
:1000800008341034FF343E34413441344134BE34FA
:100090007F3409340934093486341E342134313430
:1000A0002134DE347F34093419342934C6342634FB
:1000B000493449344934B234013401347F34013491
:1000C00081343F34403440344034BF340F34303412
:1000D000403430348F343F34403438344034BF34CB
:1000E0006334143408341434E33403340C3470347B
:1000F0000C3483346134513449344534C33442348C
:100100007F34C0347234493449344934C6342234DB
:10011000413449344934B6341834143412347F34F9
:1001200090342F34493449344934B1343E3449345D
:1001300049344934B23401347134093405348334D8
:100140003634493449344934B63426344934493490
:100150004934BE34803480348034803400344034B8
:10016000403440344034C0348207F434AD34013478
:1001700006340B341034153419341D34223427342A
:1001800028342C34313435343C34413446344B3407
:10019000503455345A345F34643469346E347334B3
:1001A00078347D34803485348A348F34943499346F
:1001B0009E34A3344134A834EE3400000000000023
:1001C000000000008316003085000030860080307B
:1001D00081009B0183128501860107309F00223038
:1001E000A00020088400A10121088000A00A2008A6
:1001F0007E3A031DF128A80A7F3083169B001C1449
:100200001A088312AC009B01AC2A003400000000E5
:10021000000000000000000000340130A400A30B27
:100220000F29A40B0F290034A30B1429A40B1429A4
:10023000003401308500062100308500062100349D
:10024000D001D101D201D301D401D501D601D7010A
:10025000D801D901DA01DB01DC01DD01DE01DF01BA
:100260000034F60CB00DF50CB00DB00DF40CB00D63
:10027000F30CB00DF20CB00DF10CB00DF00CB00D94
:10028000FE0CB10DFD0CB10DFC0CB10DFB0CB10D54
:10029000FA0CB10DF90CB10DF80CB10DF70CB10D54
:1002A0000034613084006008003A031D00342D08DA
:1002B00083169B001C141A088312AE002E08B4206B
:1002C000A90029080120A00081302002031871290B
:1002D000003020060319712920088000840AA90A29
:1002E000612920088000840A00308000AD0A2D08B2
:1002F0002C06031D0034AD0100345008F0005108F5
:10030000F1005208F2005308F3005408F4005508B5
:10031000F5005608F6005708F7005808F800590885
:10032000F9005A08FA005B08FB005C08FC005D0855
:10033000FD005E08FE005F08FF0000340730B200D9
:10034000312100308600301C192130088500310829
:1003500086000D218501B20BA029003483162030C0
:1003600085008312013085000621003085000621BA
:10037000851A0034B2291830A000513084000008DA
:1003800084038000840A840AA00BBF290034AE21B4
:1003900019217D219E2100348316FF308600003014
:1003A0008100831200000608B000831680308100AF
:1003B000003086008312301CE729B01C132A301D40
:1003C0003F2AB01D742A301E852AA7010034A718C1
:1003D0000034A714A80AD801D901DA01DB01DC0135
:1003E000DD01DE01DF012808B420A900EE3A031D7B
:1003F000FD29A801A80AA701E72958308400290887
:100400000120AA0081302A0203180B2A2A08800042
:10041000840AA90AFF292A088000840A280883166A
:100420009A0083120034271900342715A803D80135
:10043000D901DA01DB01DC01DD01DE01DF01280881
:10044000B420A900F43A031D292A2630A800A701E8
:10045000132A5830840029080120AA0081302A027A
:100460000318372A2A088000840AA90A2B2A2A0896
:100470008000840A280883169A0083120034A71982
:100480000034A7152C0883169B0083129D22831627
:100490009B0A26309A0083129D222C0883169A000C
:1004A0009A0A7F309B0083129D22AC0AD101D201AF
:1004B000D301D401D501D601D701513084002808D9
:1004C000B420A90029080120AB0081302B020318B9
:1004D0006E2A2B088000840AA90A622A2B08800051
:1004E000840AA801E7210034C72119211921192103
:1004F0000A30BA007D219E211921CC211921192110
:10050000BA0B7A2ABB215121782AA71A0034A716E0
:100510002C0883169B0026309A0083129D22AC0380
:1005200000302C060319AC0A2C0883169A007F3081
:100530009B0083129D22AD01003483161C1555309B
:100540009D00AA309D009C1483128C1FA52A8C1339
:1005500083161C1183120034C72119211921192176
:0E0560007D219E211921CC2119211921B02ABB
:02400E00503F21
:02420000260096
:0242FE000100BD
:00000001FF
